:10502A00003F0006005B004F0066006D007D000730
:10503A00007F00670077007C009300E50005000010
:103B2F0001220001240041066C01C100C103C10143
:103B3F00C10242065300004107040041071600412D
:103B4F0007000041070100012E0001230001290099
:103B5F004107120044066F000000004406F3000006
:103B6F0000004106600044072A00000000410710D2
:103B7F000041065F004207020000420714000048A0
:103B8F00072E000000000000000041070702042A72
:103B9F007FFFFFFF0425000786A34107130041069F
:103BAF00490048063D0400071D0CA7167E42064536
:103BBF000000420647000042064A000042064C0041
:103BCF000045064E0001020300420736000042077F
:103BDF00270000420705000042066D000046070857
:0A3BEF00303731363534410711003C
:10145D00FF900919122697E92408F9E43AFA0222B5
:10146D0042AF2EEF3395E0FE7C007D0B1222EF7420
:10147D008D2FF974053EFA7B01224F1222BB900984
:10148D003212269790000802225B122697900007D1
:10149D0012225BC4540325E0242EF582E43407F5B3
:1014AD0083E0FEA3E0FFE4FCFDFB7A04F9F81224CF
:1014BD004C90088B12263E90088B1225F1E47BE8A8
:1014CD007A03F9F81224D790088B12263E90088BD8
:1014DD00E47FFF7EFFFDFC1225FDD30225A6AF2E76
:1014ED00EF3395E0FEEF25E0FFEE33FE22640112AF
:1014FD0022BB90093202269790088F1226979000F2
:10150D000902225B74672FF58274053EF583A3E013
:10151D00C4F8540FC868FF05822212269790000761
:10152D0012225B1313540325E0242EF582E43407B5
:10153D00F583E0FEA3E0FF227A04F9F812244C9023
:10154D00091F12263E90091F0225F190088F1226C1
:10155D009790000702225B90089512269790000243
:10156D001223ADFFAEF022FF2479F58274063EF50D
:10157D0083EDF074792FF58274063EF583E0FF90CC
:10158D00059275F00BEB12267BEA75F00BA4258303
:10159D00F5832290091C7C007D05E0FEA3E0FF028F
:1015AD002301E4FFFEFDFCD3AB2DAA2CA92BA82A09
:1015BD00022590900895122697900002EE8FF0026A
:1015CD002404FDE0FAA3E0FB25E0FFEA33FE749E60
:1015DD002FF58274073EF583ECF0A3EDF022C413D2
:1015ED005401FFE52EFD3395E0FC74172DF5827443
:1015FD00073CF583EFF02290088F12269790000A92
:10160D0002225B900895122697122382FFAEF022DC
:10161D00E05438FF900919022697900849FDFC12F5
:10162D0025FDD3022590E0FF75F00A1222209008C7
:10163D00C6F0EF75F00A022220E0FEA3E0FFE4FC05
:10164D00FD22900895122697EE8FF00223E5900962
:10165D00150225F190097512269790000402225B60
:10166D001582E0C454F048FE2290089BE0FEA3E0F2
:10167D00FFC32212244C8F288E278D268C252212F3
:10168D00269790000612225B543F22FF131313542A
:10169D001FFEEF54C7FFEE045407FE33333354F8E7
:1016AD004F0222BB90089BE0FCA3E0FD25E0FFEC80
:1016BD0033FE22AF22EF3395E0FEEF780322E52DC6
:1016CD009528FFE52C9527FEE52B9526FDE52A951A
:1016DD00258F2D8E2C8D2BF52A2290091F12263E3B
:1016ED00E47FFF7EFFFDFC22F9F812244C90083FA9
:1016FD0012263E90083F22AF2EEF3395E0FE741771
:10170D002FF58274073EF583E05401C43354E0FF96
:10171D0022900729E0FF90092CE06F22247AF582B0
:10172D0074063EF583E022900935EEF0A3EFF0D379
:10173D00E49FE49E222473F974063EFA7B0102268F
:10174D00B790089BA3E0FF74017E00A807082290C4
:10175D00089BE0FEA3E090059475F00B12267BEE3E
:10176D002290089B12263E90089B0225F1FFEE3336
:10177D0095E0FDFC0225FDEF9408EE648094802237
:10178D00FFED64015401FE22EF3395E090089BF0CC
:10179D00A3EFF022C3135403640322AF28AE27AD89
:1017AD0026AC252290065FE0FFD36480F8229008D6
:1017BD0098122697900004229008C874FFF09008A4
:1017CD00C7F09008C6F09008C5F022900884E0C4D8
:1017DD00F8540FC86822E47BE87A03F9F80224D79D
:1017ED00E0FFD3648094809008E122E475F001025B
:1017FD00235690066CE0640122900935E0FEC3EE9D
:10180D002290089CE0940490089BE06480948022D0
:10181D003EF583E0F59BE4FFFE2274672FF582749D
:10182D00053E2290089CE025E0FF90089BE033FEEA
:10183D002290064AE0FEA3E0FF22FDE52EFB339544
:10184D00E0FAEBAE02780322E0FFA3E09006F7CFBB
:10185D00F0A3EFF022E0FFA3E09006F9CFF0A3EFA5
:10186D00F022E0FFA3E09006FBCFF0A3EFF0229073
:10187D000526E0540722FFE4F0A3EFF022752DFFBB
:10188D00752CFF752BFF752A7F223EF583E0131310
:10189D00540322EF3395E0FEEF24EBFFEE34FF22ED
:1018AD0090089BE0FCA3E0540725E0FF2253A0F72E
:1018BD0043A0102243A00853A0EF22FFE4FEFDFC3D
:1018CD00EF229008C5AFF0EFF0A3E0229008C674A8
:1018DD00FFF09008C5740AF022D3EF648094802243
:1018ED0074BE2FF58274072274FFF52DF52CF52BA0
:1018FD00752A7F22900883E0FCA3E02274272FF540
:10190D008274052274472FF582740522E49008B77E
:10191D0002263E1313135401FDEF22742E2FF58270
:10192D0074073EF58322F4FFEEF4FE3395E0FDFCE3
:10193D00225438FFE054C7225407FFE054F8229098
:10194D00000102225B1313135407FF2275BCF9909B
:10195D0007072290084902263EFFEEF0A3EFF02282
:10196D00FBEDAE047803221226B7900660E0640109
:08197D00227B017A0879C522E2
:101A3C0075FFDE75FFADE4F5E6F5E7C2AF125113A5
:101A4C00900729EFF090067312185590067512182E
:101A5C006290067712186FE4A3F0A3F0A3F0F5845C
:0E1A6C00124224124B6512509E124DF4E4FFFC
:101A7A0075F002EF90052712267BE0FDA3E090099E
:101A8A0031CDF0A3EDF0900931E0FCA3E0FDEF25A4
:101A9A00E0249EF582E434071215E3EF25E02438AA
:081AAA00F582E434071215E394
:0D1AB2000FEFB433C343E602D2AF1250E78A
:0D1ABF00124A78900931EFF0700302200AFE
:101ACC0012146EA31226B7900931E01226C01B2007
:101ADC00011B5A021B85031B8B041B91051BC7069C
:101AEC001C75071D9C081DA6091E110A1E310B1E14
:101AFC00830C1EE00D1F5C0E1F740F1F90101FAB8C
:101B0C00111FCE121FFD132002142007151FF116F2
:101B1C000000200AE524700302200A1214FF12159B
:101B2C000B1217A16019121464FFC4135401FDEFBA
:101B3C0054DF12178DC43354E01214871215EB12B4
:101B4C00148B5420FF900669E054DF021E0DE5242F
:101B5C00700302200A900932121461FFC412192179
:101B6C0054BF12178DC4333354C01214875440FF22
:101B7C00900669E054BF021E0D12504A02200A1250
:101B8C0051E702200AE524700302200A1214FFE92F
:101B9C00240A121467121698EEC39405400E121400
:101BAC00FFE9240A12146754C71222BB1214FF1245
:101BBC00160A90066B12193E021E0DE524700302E4
:101BCC00200A1214FF12155E5407600BE924071249
:071BDC00146754F8021C63BA
:101BE3001214EB74DE2FF58274073E12153D1217A3
:101BF30034501BC3E09499900935E09401500F12BF
:101C030014FFE9240712146754F844018052900921
:101C130035E0FEA3E0C39499EE94014014EE9408DA
:101C2300500F1214FFE9240712146754F84402807A
:101C33002F900935121679EE94084017EF9465EE4C
:101C4300940E500F1214FFE9240712146754F8443A
:101C530003800D1214FFE9240712146754F8440497
:031C63001222BB8F
:101C66001214FF12155E900668121945021E0DE544
:101C760024700302200A1217FF6003021D1E1214AD
:101C8600FF12155E1313135407600BE92407121491
:061C96006754C7021D0A9D
:101C9C001214EB749E2FF58274073E12153D121729
:101CAC00345018C3900935E09440500F1214FFE9DA
:101CBC00240712146754C744088043121806944032
:101CCC004014EE9480500F1214FFE924071214678D
:101CDC0054C74410802812180694804014EE94C007
:101CEC00500F1214FFE9240712146754C7441880CC
:101CFC000D1214FFE9240712146754C74420122252
:011D0C00BB1B
:101D0D001214FF12155E90066812193E4FF0021F55
:101D1D00A912148B5407600812146454F8021D8B19
:101D2D001214EB1218ED3E12153D1217345015C357
:101D3D00900935E09440500C90093212146154F81A
:101D4D004401803A12180694404011EE9480500CD4
:101D5D0090093212146154F844028022121806942C
:101D6D00804011EE94C0500C90093212146154F859
:101D7D004403800A90093212146154F8440412226B
:011D8D00BB9A
:101D8E0012148B9006691219454FF0021FA9900587
:101D9E0025E06401F002200AE524700302200A12F5
:101DAE0014FFE92409121467FFC313FEEF54F9FF61
:101DBE00EE045403FE25E04F1222BBEE6403700DB9
:101DCE0012148B1215EB121464442080201214FF8F
:101DDE0012150BC313540370171217041214645404
:101DEE00DF4F1214FCE9240912146754F91222BBB6
:101DFE001214FF12150B5406FF90066AE054F94FA9
:101E0E00021F8D90066CE0FFC374039FFFF0BF01AD
:101E1E000590066F80039006F312264AFFFFFFFF20
:101E2E0002200AE524700302200A1217FF900932DD
:101E3E007021121461FF12192054F712178D3333CB
:101E4E003354F81214875408FF900669E054F74F84
:101E5E00F0801F121461FFC45401FDEF54EF1217EE
:101E6E008DC454F01214875410FF900669E054EF9D
:101E7E004FF0021FA9E524700302200A1217FF90EB
:101E8E0009327023121461FFC4121920547F1217E5
:101E9E008DC433333354801214875480FF900669F7
:101EAE00E0547F4FF08028122697E9240912146718
:101EBE00FF5401FDEF54FEFFED640154014F121467
:101ECE00FC12150B5401FF90066AE054FE4FF0020F
:101EDE001FA9E524700302200A1217FF7033121493
:101EEE00FFE92409121467121698EED39406400ED9
:101EFE001214FFE9240912146754C71222BB1214DC
:101F0E00FF12150B5438FF90066AE054C74FF0804D
:101F1E003B1214FFE9240A121467FF54F8FEEF0473
:101F2E005407FF4E1222BBEFC39407400E1214FF4C
:101F3E00E9240A12146754F81222BB1214FF121667
:101F4E000A5407FF90066BE054F84FF0804DE524DD
:101F5E00700302200A1214FF1222421214FA1222E5
:101F6E00429006618019E524700302200A1214FFC4
:101F7E00E924011214671214FA12194C900662F039
:101F8E00802E900526E0FF54F8FEEF045407FD4E18
:101F9E00F0EDC394034004E054F8F08013E52460A0
:101FAE0014900660E004F0C3648094834002E4F071
:101FBE0012513B80477524019006607401F0803CFD
:101FCE0020000EE4900524F0121A33C203C20280E0
:101FDE002BA201B39201300106C206D202801DC2AD
:101FEE00028019900729E0FF7D1C1250FD800D63C1
:0C1FFE002401800812198580031247E6B8
:10200A00124E62EF7003021ABF90092BE0FFB40B65
:10201A0002D200EF6431701412171E700F1220DE04
:10202A00A3E09008D5F01242FB1220F490092BE0AD
:10203A006432700E12171E70091220DE1243B1129A
:10204A0020F490092BE0642D700E12171E700912ED
:10205A00210412464E12211A90092BE0642E700EAA
:10206A0012171E700912210412446712211A9009CC
:10207A002BE030E7097B017A09792A124E929009FE
:10208A002BE0FFB41406D201D202C206EFB4150443
:10209A00C201C202200103021ABFEF14601E0460CB
:1020AA0003021ABF90092CE0FFC3941E4003021AD0
:1020BA00BF900524EFF0124DF4021ABF90092CE0EC
:1020CA00FFC3941E4003021ABF900524EFF0121AB0
:0420DA0033021ABFF4
:1020DE001251C27F327E0012514E90092DE0FFA3A5
:1020EE00E0FDA3E0FB227F327E0012514E900729C5
:1020FE00E0FF121A21221251C27F327E0012514E7F
:10210E0090092DE0FFA3E0FDA3E0FB227F327E00CD
:0C211E0012514E900729E0FF121A2122F6
:1051130030B60930B7037F41227F422230B7037F85
:0551230051227F522221
:10422400900912E584F075FFDE75FFAD75840F7596
:054234009601758C20CD
:10423900E4A3F0A3F09009131216467B407A9CF987
:0F424900F8D312259040089009131217F880E659
:10425800E4F58475EF0675840F758A83F597758480
:104268000F758904F58475B73075840F4389017516
:104278008D01758F01758E0490090E12264A000073
:104288000000E4FF7E01FDFC90090E1225FDC3121B
:1042980025A6501B90090E1225F1EF2401FFE43EDC
:1042A800FEE43DFDE43CFC90090E12263E80D3431B
:1042B8008902E58920E41290090E122609E4FB7AA6
:1042C80001F9F8C31225A650E9759702E4F58A901A
:1042D8000912E0F584E4F584124F731250841251E8
:1042E80072124D421251DD125182124C7D90090E0C
:0342F80002263E5D
:104F730075840F75A4CF75A71C75B0E7E4F5E275CA
:104F8300A6FF75E10375E3C0F5A57590FF75ADE365
:084F930075AD63F5A5F584225C
:10508400E4F58443E60875DA3175DB3175DC317596
:0A509400DD3175D983D2DEF58422E8
:10517200D2AF759A4075F809759D01C286C2872221
:0A51DD0075E8C075BCF875D1032217
:10514E00E4FDFCC3ED9FEC9E50070DBD00010C80ED
:01515E00F25E
:01515F00222D
:1051820075840275E88075BCF975D103E4F5842253
:104C7D00AB84E4F584F588758DF0F58B758910F5A9
:104C8D008E75884090095912264A0000F00DE4F502
:104C9D008475CC0D75CDF075CA0D75CBF0F5C97554
:104CAD00C80443A82843B808AF038F84900959124C
:024CBD0025F1DF
:014CBF0022D2
:1050E700E4F5BB758402900707E0F5BBE4F584435C
:0650F700E71243F712224C
:10504A00AF22121470900526E04408F012160A12D4
:0D505A0019526003BF04061245B41218F588
:015067002226
:0851E700900526E054F7F022C8
:1045B40012168FFF7005E522048007121667700932
:1045C400EF1490095DF00246391216C0C333CE339E
:1045D400CED8F9FDAC062479F58274063CF583E067
:1045E400D364809480401712168F1490095DF07480
:0E45F400792DF58274063CF583E014F08037D3
:10460200AF2212147090095E1226B7E522049009B7
:104612005DF01216679000051222CD90000512225D
:104622005BFD1216C0C333CE33CED8F92479F5829E
:0746320074063EF583EDF074
:1046390090095DE0C3648094904002E4F090095DC4
:05464900E0FF024EF14C
:104EF1008522238F229006FD7401F0A3F0A3F0EF29
:104F01003395E0FE90059775F00BEF12267BEE12BC
:0D4F11001597E0121952BF04031251E72258
:1051280012187CFFBF010B900713E0FF124EF1121B
:0351380018F52245
:031A39000226E69C
:1026E600C0E0C0F0C083C082C0D075D000C000C0BA
:0D26F60001C002C003C004C005C006C0073B
:10270300758402C2ED90083AE5BEF0900707E02415
:10271300FD70030227A1147003022B4A24FD7003EA
:10272300022B6924056003022BC590083AE0900848
:10273300021218837D327F321238A7900713E0907C
:102743000649F0900702E0C4540FFD90058BE0C4E6
:10275300F854F0C8A3E0C4540F482D900713F0D3E6
:10276300940F4004E024F0F0900649E0FE90071334
:10277300E0FFB506046522600D12187CFEBE02065A
:10278300124EF112188A900649E0FF900713E06F8A
:0E279300600312513B1219597403F0022BC55A
:1027A10090071412164690085112263E90085712AF
:1027B100264A0000016390085B12264A00071C00AC
:1027C100AF2212147090085F1226B7E522FD3395EF
:1027D100E0FCED1216B9121511D58202158315828E
:1027E100E0C454F048900845F0A3EFF012155E5490
:0327F10007602D51
:1027F400EDAE047803C333CE33CED8F9121729C40F
:102804005403FF900862F01214EE121928E0C4F881
:0B28140054F0C868FFA3E0C4540F4854
:10281F00800EAF221214ED121827F583E0FFA3E00C
:10282F00900847CFF0A3EFF0900847E0FCA3E0FD3E
:10283F00EC1313543F90083EF0EC5403FEAF05E445
:10284F00FCFDA31216FD1225F1E47B637A0112162B
:10285F00F51225FDC3E49BFF74A89AFE740C99FD35
:10286F00E498FC90083F12263E90083EE025E024B5
:10287F003DF582E4340612153D90083BEEF0A3EFD0
:10288F00F0FBAA06E4F9F890083F1225F11224D7BD
:10289F00121960900704E4F090085F12148EFFC4C1
:1028AF0013540720E0030229E212150B1217A1603F
:1028BF00030229441214EB12182712153DC3941664
:1028CF00EE9401500AEF94A4EE94004002805DC391
:1028DF00EF94FFEE9402500AEF94B9EE9402400287
:1028EF00804AC3EF94A7EE9406500AEF94F8EE9443
:1028FF000540028037C3EF94EBEE9408500AEF9433
:10290F0095EE940840028024C3EF9417EE940C5078
:10291F000AEF94D1EE940B40028011C3EF945BEE5B
:10292F00940F500EEF94E9EE940E40069007047446
:10293F0001F00229E2E47FC77E01121627400C90B6
:10294F00084D12264A000002808031E4FF7E0112FA
:10295F001627400C90084D12264A00000140801C9B
:10296F00E47F8FFE12162790084D400912264A0069
:10297F000000A0800712264A00000050900845E092
:10298F00131313541F7E00121966C3941CEE940088
:10299F0050047F0180027F00900845E0FCA3E0FD1A
:1029AF00D39404EC940040047E0180027E00EE5F1D
:1029BF00602D7E00ED54079008451219666407607C
:1029CF000A900845E07002A3E070149007047401A8
:1029DF00F0800C9008491225F190084D12263E7F89
:1029EF00A37E867D077C0090084D1225FD12168070
:1029FF0078081225CA12168390085F121508C313A0
:102A0F005403601024FD600C240270141217A8E404
:102A1F007B0880061217A8E47B40FAF9F81216809B
:102A2F0090083AE09007FE1218837D307F301238FD
:102A3F00A790083DE0FF90070EE4F0A3EFF090059C
:102A4F0087A3E090083DF0900589E0FFA3E0900890
:102A5F0055CFF0A3EFF090085574FF75F080122357
:102A6F0056900855E0FEA3E090085112177A1224F1
:102A7F004C1219609008491225F1780F1225CA12CD
:102A8F00196090083DE0FFE4FCFDFE900849122517
:102A9F00FD12243190084D12263EE47FFFFE900870
:102AAF004D12162A400A90084D12264A000000FFC8
:102ABF0090084D1225F1EC33500A90084D12264A1A
:102ACF000000000090084D1225F190083DEFF0E056
:102ADF00FFC413135403A3F0EF543FFFE4FCFDFEB8
:102AEF00A31216FD1225F1E47B08FA1216F5122532
:102AFF00FDC374F89BFF74039AFEE499FDE498FC00
:102B0F001216FA1225F190083EE0F9F81225B79047
:102B1F000843EEF0A3EFF01217A878081225CA1297
:102B2F001683AB28AA27A926A82590084312164674
:0B2B3F001216801219597404F0807BFC
:102B4A0090083AE0FF900800E4F0A3EFF07D317FAF
:0F2B5A00311238A775BCF89007077407F0805C3C
:102B6900900645E0FEA3E0FFA3EEF0A3EFF0900886
:102B79003AE0FD900645E4F0A3EDF0D3EF9480EE42
:102B89009400500EE09480900645E09400400312B2
:102B9900504AD3900646E09425900645E0940050AB
:102BA90008E50B5404FFEF70089007167401F080D4
:0C2BB90005900716E4F01219597402F0A0
:0C2BC500900707E0F5BB75840043E810A2
:102BD100D007D006D005D004D003D002D001D00058
:0B2BE100D0D0D082D083D0F0D0E03202
:031A3000020C9A0B
:100C9A00C0E0C0F0C083C082C0D075D000C000C020
:0D0CAA0001C002C003C004C005C006C007A1
:100CB700AF2212147090088F1226B7AF23EF339527
:100CC700E0FE1222EF748D2FF974053EFA90089218
:100CD7001226B71216C0C333CE33CED8F990089573
:100CE700121742AF231216C2C333CE33CED8F990B0
:100CF7000898121742C2EDE4FFFEFDFC90072A1286
:100D0700162C401590072A1225F174FFFBFAF9F803
:100D170012243190072A12263EE47F01FEFDFC9043
:100D2700072A1225FDC3122590700D12512890072E
:100D37002A12264A00000000AFBFEFFFADBEED90BC
:100D47000883CFF0A3EFF01217B174809840030225
:0D0D57000ED4C3EF648094904003020ED4CC
:100D64001217951217FF707812190190089B12152B
:100D7400CFAF031217548005C333CE33CED8F990C6
:100D8400066F12177A122569EC4D4E4F604A1218FD
:100D940030749E2FF58274073EF583E0FCA3E0FDDA
:100DA40074382FF58274071215E290066F1225FD30
:100DB400C000C001C002C00312174E8005C333CE69
:100DC40033CED8F9121933D003D002D001D0001297
:100DD400256990066F12263E90089BA3E0020E6DD3
:100DE400121901FD90089BE0FAA3E0FB25E0FFEA5D
:100DF40033FE1218ED1215E2AF031217548005C327
:100E040033CE33CED8F9FFEE3395E0FDFC9006F3F4
:100E14001225FD122569EC4D4E4F60461218301212
:100E240018ED3EF583E0FCA3E0FD74582FF58274C1
:100E3400071215E29006F31225FDC000C001C0029E
:100E4400C00312174E8005C333CE33CED8F912191E
:100E540033D003D002D001D0001225699006F312DA
:100E6400263E90089BA3E02410FDFF1238A712171A
:100E74005C121597E01313135407601A1216B1127B
:100E8400190912189712196DC333CE33CED8F9123B
:100E9400172954FC4BF090089BE0FEA3E0900595C5
:100EA400121766121597E054077003020FD6121634
:100EB400B1121911121897FF25E025E012196DC31C
:0D0EC40033CE33CED8F912172954F34BF07A
:0B0ED100020FD690065FE06410702D49
:100EDC001217D8FF90088312166FE4FCFD12176EE0
:100EEC00E4FB7A04F9F812244C12176E1217E31271
:0A0EFC00176E900702EEF0A3EFF06E
:100F0600020FD61217B17411648098500EC3EF64A5
:050F16008094955006D7
:030F1B00EF24EFD1
:100F1E00020FB71217B174156480985054C3EF6462
:050F2E008094A5504C69
:100F33001218A0FE1217992420FFE43EA3F0A3EF9A
:100F4300F012190190089D1215CFAD03AF051238A9
:100F5300A712175C121597E0540760771216B112A7
:100F63001827121898FFC454F012196DC333CE33E7
:0A0F7300CED8F912172954CF4BF025
:100F7D00805790065FE0FDB425151217D8FE900836
:100F8D0083E0C454F048900714F0A3CEF0803AD318
:100F9D00ED6480F87426648098502E90065FE0FF13
:070FAD00C3648094AA5022E6
:100FB400EF24DAFF90089BF0FD1217D8FB9008830A
:100FC400E0C454F048FAED1214EE121928EAF0A322
:020FD400EBF040
:100FD60012155813131354076017900525E0702750
:100FE60090089512155B12153212150512143C80E5
:100FF60013AF221214ED121909121518D582021513
:101006008312166D12164F90089212155B13131366
:101016005407601A900525E0702D90089812155B0C
:101026001215329008921215081214488013AF2335
:101036001214ED121909121518D58202158312160B
:101046006D90089812165290088F12148E540760ED
:1010560014900525E07024900895121527121604A1
:101066001214548013AF221214ED1219111215180E
:10107600D58202158312166D1215C09008921214AD
:101086008E5407601C900525E0702F900898121565
:10109600279008921216075407FDAB23123F638070
:1010A60013AF231214ED121911121518D582021559
:1010B6008312166D9008981215C3121558540760BE
:1010C60020900525E07033900895121497400A90F9
:1010D600088B12264A0000FFFF90088B1225F1802C
:1010E60010AF221214ED121511D5820215831216B5
:1010F6006D9008951217BE1215C990089212155BCD
:1011060054076020900525E07030900898121497D7
:10111600400A90088B12264A0000FFFF90088B12A7
:1011260025F18010AF231214ED121511D582021588
:101136008312166D1217BB1215C912155813131305
:101146005407700C12161012150512143C12164F85
:1011560090088F12148E5407700C12156412160420
:101166001214541215C0900700E4F090088F121460
:101176008E131313541F30E014121610124ACB901C
:101186000700EFF0121610124BAD12164F90070122
:10119600E4F090088F12148EC4540F30E014121528
:1011A60064124ACB900701EFF0121564124BAD1290
:1011B60015C090088F12148EC4131313540130E017
:1011C6003D900898121613900892121508121448AA
:1011D600900898121652121610E4FCFDC004C005C1
:1011E600C006C007900898121613121919D007D016
:1011F60006D005D004124948900885EE800F900865
:1012060095122697122382FF900885E5F0F0A3EF4A
:10121600F012150530E04290089812156790089272
:101226001216075407FDAB23123F63900898121558
:10123600C3121564E4FCFDC004C005C006C00790D7
:101246000898121567121919D007D006D005D004D0
:10125600124948900887EE801290089512269790BA
:1012660000021223ADFF900887E5F0F0A3EFF0909F
:10127600088F12148EC41313540390089530E02B74
:101286001217BE12156DE4FCFDC004C005C006C0F1
:10129600071217BB12156D121919D007D006D00503
:1012A600D004124948900889EE800C1217BE12230A
:1012B600ADFF900889E5F0F0A3EFF09008851218CD
:1012C6005590088712186290088912186F900710B7
:1012D6001217B4748098505DC3EF64809490505593
:1012E6001217951218ADA3EFF0C3EC6480948040FA
:1012F6000A12180E50051218BA80141216769404A3
:10130600EE64809480400E12178450091218C1753D
:10131600BB000213CE121676121785400FEF940CFF
:10132600EE6480948050051218BA80031218C175B5
:02133600BB01F9
:101338000213CE900710E0FFB4100675BB0202142A
:1013480008EFB411030213EAEFB412030213F3EF28
:10135800B413030213FCEFB41403021405D3EF64AF
:1013680080F874156480985068C3EF648094A55021
:011378006014
:101379001218A01217991218ADEF04A3F0C3EC6468
:10138900809480400A12180E50051218BA8014125F
:1013990016769404EE64809480400D1217845008E8
:1013A9001218C175BB00801D121676121785400FE1
:1013B900EF940CEE6480948050051218BA800312E1
:0E13C90018C175BB0153A0F890089DE042A02A
:1013D700802F900710E0FFB4250575BB038022EF2F
:1013E700B4260575BB048019EFB4270575BB0580C6
:1013F70010EFB4280575BB068007EFB4290375BB4A
:1014070007900710E090065FF090071004F0C364A0
:0A1417008094AA4002E4F012371A94
:10142100D007D006D005D004D003D002D001D0001F
:10143100D0D0D082D083D0F0D0E032131313540730
:10144100FDAB22123F63221313135407FDAB23128A
:0C1451003F63225407FDAB22123F6322D0
:104FC200EF252EF52ED36480948F4003E4F52EC393
:104FD200E52E648094805003752E0FE52460031241
:034FE20031E92290
:1031E900AF0BAE0AAD09AC0812258390091512265A
:1031F9003E12146E9009191226B712165BEF54018C
:103209001218C8600F900669E0542012145D54DF4B
:103219004F1222BB12165BEF54021218C8600F90AE
:103229000669E0544012145D54BF4F1222BB1216B6
:103239005BE4FFEE5401FEE4FDFCEE604890066A93
:10324900E01217A1701090091912148E1215EB12C1
:10325900146444208017900919121508C3135403E4
:10326900FFBF030C12170412146454DF4F1222BB60
:1032790090066AE05406121620E9240912146754CC
:10328900F94F1222BB12165BE4FFEE5404FEE4FD73
:10329900FCEE602090066CE0900669B4010AE054E7
:1032A9000812145D54F78008E0541012145D54EFAD
:1032B9004F1222BB12165BE4FFEE5408FEE4FDFC3C
:1032C900EE602990066CE0B4010D900669E0548027
:1032D90012145D547F801190066AE0540112162081
:1032E900E9240912146754FE4F1222BB12165BE43B
:1032F900FFEE5410FEE4FDFCEE602C90066CE0B489
:10330900011090066A12161DE9240912146754C7A0
:10331900801190066BE05407121620E9240A121452
:103329006754F84F1222BB12165BE4FFEE5420FEDD
:10333900E4FDFCEE600B900661E0121620EF12220C
:10334900BB12165BE4FFEE5440FEE4FDFCEE600E9A
:10335900900662E0121620900001EF1222CD12169B
:103369005BEF54401218C8602690066CE0B4011057
:1033790090066812161DE9240712146754C7800BBA
:10338900900669E0540712145D54F84F1222BB12DB
:10339900165BEF54201218C86012900668E05407B3
:1033A900121620E924071214671216AB12165BEFE6
:1033B9005410FFEF601290066B12161DE9240A12D1
:0833C900146754C74F1222BB28
:0133D10022D9
:053C560090093AEDF0B9
:103C5B0090064C1217F8FED3E5F0121785401BE4C3
:103C6B0090064CF0A3F090064A1217F9FEE5F064AB
:103C7B00044E700690064AF0A3F012183E64034EF1
:103C8B006006EF64014E702290064CE0FEA3E0FF4D
:103C9B004E700990064CF0A304F0800EEF64034EB7
:103CAB00700890064CF0A37407F012183E2404FD24
:103CBB007401A805088002C333D8FC90065AF0C3E0
:103CCB0090064DE0940890064CE064809480505927
:103CDB008F828E8312225BFF90093CF01214EE74DC
:103CEB002A2FF58274503EF583E493FC740193FD07
:103CFB0090064CA3E0FB74017E00A803088005C36B
:103D0B0033CE33CED8F9FFEC5EFEED5F4E600890FC
:103D1B00065AE02BF08005E490065AF090093CE03F
:073D2B00C364809480503353
:103D3200802C12183EEE702BEF14600A14601114DE
:103D4200600E2403701D90093BE060028008800E23
:103D520090093AE0600890065AE02407F022E490C5
:033D6200065AF00E
:013D6500223B
:0447E600E5246072F4
:1047EA0012146E90097512197470239009751216B5
:1047FA008CD394004012E92406121467FF54C0FEB9
:10480A00EF14543F4E1222BB12513B0248599006F4
:10481A0060E064027034121661FFD36480948140B0
:10482A000A90000474FF122288800BEF700890002F
:10483A000474131222CD121661121847C333CE33F1
:10484A00CED8F9121574EFF080057FFF124FC2021D
:02485A00513BD0
:06485C007FFF124FC22293
:04198500E524607B7A
:1019890012146E9009781219747020900978121641
:101999008CC394105012E92406121467FF54C0FE38
:1019A900EF04543F4E1222BB0219F7900660E0641F
:1019B900027040900978121664FFC36480949350B2
:1019C9000DEF600A9000047401122288800BEFB4B5
:1019D9001307900004E41222CD90097812166412BC
:1019E9001847C333CE33CED8F9121574EFF012511C
:0B19F9003B80057F01124FC202513BF2
:061A04007F01124FC22217
:031A12000251D1AD
:0C51D100C2CF75840243E81075840032E0
:10358A0090066CE0B40107900700E0FC8005900704
:10359A0001E0FC12150BC3135403FF64036015907A
:1035AA000655E0FE7401A807088002C333D8FC4E12
:1035BA00900655F0900658E0FF122242FEEF4E9018
:1035CA000658F0E0FF12194C25E0FEEF4E9006581F
:1035DA00F0121491FEC413540730E013900704E06C
:1035EA009006556006E04410F08004E04420F09014
:1035FA000655E0FFEEC41313540133333354F8FE77
:10360A00EF4EF090066CE0900656B4010BE0FF1204
:10361A001491C41313138005E0FF12150B5401FE15
:10362A00EF4E900656F090066CE0FF64017013129C
:10363A001491131313541F30E021EC9006566017AF
:10364A00800F121491C4540F30E010EC90065660AB
:10365A0006E04402F08004E04404F0EFB4010812EA
:10366A00150B131313800312160A5407FDEDB40544
:10367A0009900657E04420F0803EED700990065705
:10368A00E04401F08032EDB40109900657E04402AB
:10369A00F08025EDB40209900657E04404F0801842
:1036AA00EDB40309900657E04408F0800BEDB4042A
:1036BA0007900657E04410F012160A1219526021B8
:1036CA00900659E0FE744E2FF582E43406F583E045
:1036DA00FF7401A807088002C333D8FC4E9006592C
:0136EA00F0EF
:1036EB0012155EFF54076007900659E04410F090E6
:1036FB00066CE0B4010AEF13131354076010800734
:0E370B0012149154076007900659E04420F014
:01371900228D
:103D6600E4900952F0A3F09009521216799405EEE8
:103D760064809480501474552FF58274063EF58342
:103D8600E4F09009521217F980DDE5246004AF2EA5
:103D96008002AF2212147090094F1226B790094F75
:103DA60012269712358A12187CFDBD010990065815
:103DB600E04404F0800ABD0207900658E04408F08B
:103DC600900656E0FF90066CE033333354F8FEEF6E
:103DD6004E900656F0300207900658E04410F090D8
:103DE6000658E0FFE524C43354E0FEEF4EF090059C
:103DF60026E0131313541F90065530E006E0448066
:103E0600F08004E04440F0900659E0FF900525E07C
:103E1600C4333354C0FEEF4E900659F0C2FA9009EF
:103E260052E4F0A37404F053F87FE59A20E7FB9080
:103E36000952E0FEA3E02455F582740612181D0F00
:103E4600BF00010EEF64324E70F590095274FFF513
:103E5600F0122356900952E0B4FFCCA3E0B4FFC79A
:023E6600D2FA8E
:013E68002237
:10371A00E49008C3F0A3F09008C31216799403EE5C
:10372A00648094805014745A2FF58274063EF5838F
:10373A00E4F09008C31217F980DDE52230E31C900B
:10374A00065CE0FFE5225407FE7401A80608800221
:10375A00C333D8FC4F90065CF0801790065BE0FFFD
:10376A00AE227401A806088002C333D8FC4F900623
:04377A005BF0C287B7
:10377E0012146E9008C91226B7AF2E1216C2C3339A
:10378E00CE33CED8F92473F974063EFA7B01900835
:10379E00CC1226B79008C912168CFF9008CFF012E3
:1037AE0016679008D0F09008CC122697900006125B
:1037BE00225B9008D112163E9008C812163E900851
:1037CE00C71218D2700374FFF0E52460559008D02C
:1037DE001216331218CF700374FFF09008CFE0FF6B
:1037EE00D3648094804007A3E070031218D9EF7061
:1037FE00031217C5900660E0B4020C12197E9009F0
:10380E003B7401F0E48018900660E012197EB4015A
:10381E0009E490093BF07D018037E490093BF0FD0F
:10382E00802F9008D11216331218CF700374FFF048
:10383E009008CFE0FF70031217C51218E6400990EA
:10384E0008D0E070031218D912197EE490093BF0EB
:04385E00FD123C56C5
:103862009008C3E4F0A37402F053F87FE59A20E7CE
:10387200FB9008C3E0FEA3E0245AF58274061218F6
:103882001D0FBF00010EEF64324E70F59008C37435
:10389200FFF5F01223569008C3E0B4FFCCA3E0B4C6
:0438A200FFC7D28703
:0138A60022FF
:10486200E4FD7C0290065DE4F0A3DCFC7C007D02AA
:10487200E52E30E31C90065EE0FFE52E5407FE7441
:1048820001A806088002C333D8FC4F90065EF08070
:104892001790065DE0FFAE2E7401A806088002C3E1
:1048A20033D8FC4F90065DF0C2A57C007D0153F821
:1048B2007FE59A20E7FB745D2DF58274063C1218A1
:1048C2001E0FBF00010EEF64324E70F5ED1D700138
:0948D2001CBCFFDABDFFD7D2A522
:0148DB0022BA
:10476800900736E0FFA3E0900727CFF0A3EFF0E52E
:10477800905440FF900736E4F0A3EFF0900705E06F
:10478800FFA3E090066DCFF0A3EFF0E5905420FF73
:10479800900705E4F0A3EFF0900727E07002A3E08C
:1047A8007015900736E07002A3E0600B900727E4CD
:1047B800F0A304F01251E790066DE07002A3E070D8
:1047C8001C900705E07002A3E0601290066DE4F00B
:0E47D800A304F090072A12264A0000003222A5
:031A0C00022F8422
:102F8400C0E0C0F0C083C082C0D075D000C000C013
:0D2F940001C002C003C004C005C006C00794
:102FA100C28FAF221214709008E31226B790071255
:102FB100E0FF2408F582E43407F583E09008E0F0AF
:102FC100EF14603914606014606F14700302305F95
:102FD10014700302308D240560030230A89006F7B7
:102FE1001216469008E612263E9008E61214DD40BD
:102FF1002A9008E612264A0000FFFF801E9006F97B
:103001001216469008E61216EA9008E61214E440F9
:103011000A9008E612264A0000FFFF9008E61225F2
:10302100F19008E1EE800B9006FBE0FFA3E0900831
:10303100E1CFF0A3EFF00230A89008E31226971237
:103041002242603F9006FE1217ED400474FF80019A
:10305100E4F0A3F01218E6404E9006FE8046900878
:10306100E312269712194C601A9006FF1217ED40D1
:103071000474FF8001E4F0A3F01218E640299006E1
:10308100FF80219008E1E4F0A3F0801B9006FD127F
:1030910017ED400474FF8001E4F0A3F01218E6403C
:1030A100069006FDE014F0C28653F87FE59A20E70A
:1030B100FB9008E0E0F59BE4FD0DEDB432FB9008D8
:1030C100E1E0FF7E0053F87FE59A20E7FB8F9B7DCF
:1030D100000DEDB432FB9008E1A3E0FF7E0053F850
:1030E1007FE59A20E7FB8F9B7D000DEDB432FBD28B
:1030F10086900712E004F0C394064002E4F0124700
:1031010068900711E024FA600924067008123D66F0
:103111008003124862900711E004F0E05407F012B6
:10312100187C6007640160030231AF1217A8C31253
:1031310015B540061216CB0231C81215AF40030275
:0A31410031BC1215AF40030231C883
:10314B009008EAE4F09008E31216071313135407E0
:10315B0024FE601114601E2402702E12150B121720
:10316B00A16026801E900716E0701E12150B121719
:10317B00A16016800E900716E0600E12150B121749
:10318B00A160069008EA7401F09008EAE0602E90C6
:10319B000526E0FF131313541F30E0211245B41220
:0231AB00188A80
:1031AD0080191215AF40031216CB1215AF500C75C6
:1031BD002D00752C00752B00752A00758DF0758B03
:0131CD000001
:1031CE00D007D006D005D004D003D002D001D00055
:0B31DE00D0D0D082D083D0F0D0E032FF
:064948009008B312263EA8
:10494E00AF2DAE2CAD2BAC2A780F1225CA9008BB1A
:10495E0012263E9008BB1225FDC3E49BFFE49AFE8F
:10496E00740199FDE498FC9008BF12263E9008B39E
:10497E001225F19008BF1225FD12244CC004C0056B
:10498E00C006C0079008B71225F19008BB1225FD8E
:10499E0012244CD003D002D001D000122431781052
:0349AE001225B718
:0149B10022E3
:104BAD007C027D8F1223017C027D8F1222EFE4FCAB
:104BBD00FDFB7A04F9F812244C90096112263E90FF
:104BCD0009611225F11217E39009611216EA900995
:104BDD00611214E4400A90096112264A0000FFFF99
:064BED009009611225F1A0
:014BF300229F
:104ACB0090097BEEF0A3EFF0C374469F74019E50E8
:104ADB003A90097B1216467BAA7AFEF9F8122590BA
:104AEB00402990097B7C027D8F1215A790097BECE6
:104AFB00F0A3EDF0C3943CEC9400400CD3E094583D
:0E4B0B0090097BE0940240037F01227F00228C
:0B3F630090091CEEF0A3EFF0A3EDF0BE
:103F6E0014601A14602314602C14603524FE604112
:103F7E00240660030240171215A002400F1215A06E
:103F8E00EF2430FFEE343380221215A0EF2460FFB1
:103F9E00EE346680161215A0EF2490FFEE34998051
:103FAE000A1215A0EF24C0FFEE34CC90091C02407B
:103FBE0013AF03E4FCFDFE12154CE47BFF7AFF12F7
:103FCE00154778041225B712154CE47B29121545B6
:103FDE00E4FB7A04F9F81224D712154CE42FFFEE05
:103FEE003408FEE43DFDE43CFC1216E790091F1276
:103FFE0014E4400A90091F12264A0000FFFF121512
:10400E005290091CEEF0A3EFF090091EE0640660DA
:10401E002D90091C121646FB1215451217E31216A7
:10402E00E790091F1214E4400A90091F12264A0055
:10403E0000FFFF12155290091CEEF0A3EFF090094D
:06404E001CE0FEA3E0FFF0
:014054002249
:105192000001FF00FF000001010000FF00FF01000D
:103BF900040800000000041A000000000416000078
:103C0900000002130000011500010D00020E000062
:103C1900031000000044086B000000004408630022
:103C29000000004208690000410867004108680077
:10451100AF0BAE0AAD09AC08022583FC9008F61278
:10452100263E9008F60225F1EF5401FFE4FEFDFC62
:10453100EF2290086B1225F1EC4D4E4F22AFB0FEE9
:10454100EF5407FFE478100225DEE4FFEE5401FE8C
:10455100E4FDFCEE22E4FFEE5402FEE4FDFCEE225B
:10456100E4FFEE5404FEE4FDFCEE22E4FFEE540809
:10457100FEE4FDFCEE22E4FFEE5410FEE4FDFCEE51
:1045810022E4FFEE5420FEE4FDFCEE22E4FFEE54B3
:1045910040FEE4FDFCEE22E4FFEE5480FEE4FDFC6F
:1045A100EE22E4FFFEED5401FDE4FCED22900966EC
:0345B10002269748
:104B6500D2B3C2B4125008E4FCFDC004C005C006AF
:104B7500C00712453ED003D002D001D000122576E1
:104B85008F198E188D178C168F1D8E1C8D1B8C1AE8
:104B9500AF907513008F147B017A08796F8B108A9B
:084BA5001189128A0E890F220A
:0549B200900965EFF023
:1049B700E50F2401FFE4350EFAA9077B01A31226B0
:1049C700B71245AE74019008836B7008E965827071
:1049D70003EA6583700C7B017A08796F9009661288
:1049E70026B71245AEE5108511838512826B7008D4
:1049F700E965827003EA65836019900965E0850FB0
:104A070082850E83F01245AEAF018A0E8F0F900993
:034A170065E0F067
:014A1A002279
:104A780053E6F7AA0EA90F7B01E51085118385126D
:104A8800826401700AE50F65827004E50E65837023
:104A980003FF802B7810E475F0011226871222425A
:104AA800FF74019008836510700AE512658270042E
:104AB800E5116583700975100175110875126F434A
:024AC800E608FE
:014ACA0022C9
:031A1E00022BECAC
:102BEC00C0E0C0F0C083C082C0D075D000C000C0AF
:102BFC0001C002C003C004C005C006C00720DF032B
:032C0C00022EF89D
:102C0F00E50C6005D50C02D20C125008E4FCFDC097
:102C1F0004C005C006C00712453ED003D002D00144
:102C2F00D0001225768F0B8E0A8D098C08AF1DAE42
:102C3F001CAD1BAC1AAB0BAA0AA909A808C3122515
:102C4F00A6602BE50B651DFFE50A651CFEE5096512
:102C5F001BFDE508651A12451CEC4D4E4F600375C0
:102C6F001503850B1D850A1C85091B85081AE5159B
:102C7F007003022E581515E5156003022E58E5193D
:102C8F00650BFFE518650AFEE5176509FDE5166595
:102C9F000812451C124529600D1245111245296075
:102CAF00057F011249B2124523EF540212452C60E1
:102CBF0010124511EF540212452C60057F02124984
:102CCF00B2124523EF540412452C6010124511EF38
:102CDF00540412452C60057F031249B2124523EFAD
:102CEF00540812452C6010124511EF540812452C50
:102CFF0060057F041249B2124523EF541012452C80
:102D0F006010124511EF541012452C60057F05120B
:102D1F0049B2124523EF542012452C601012451171
:102D2F00EF542012452C60057F061249B21245233D
:102D3F00EF544012452C6010124511EF54401245CC
:102D4F002C60057F071249B2124523EF54801245BC
:102D5F002C6010124511EF548012452C60057F082E
:102D6F001249B212452312454B600D1245111245FF
:102D7F004B60057F091249B2124523124556600D6B
:102D8F0012451112455660057F0A1249B2124523AA
:102D9F00124561600D12451112456160057F0B12DE
:102DAF0049B212452312456C600D12451112456C44
:102DBF0060057F0C1249B2124523124577600D1240
:102DCF00451112457760057F0D1249B21245231246
:102DDF004582600D12451112458260057F0E124922
:102DEF00B212452312458D600D12451112458D60AB
:102DFF00057F0F1249B2124523124598600D1245F7
:102E0F001112459860057F101249B21245231245E1
:102E1F00A3600D1245111245A360057F111249B22F
:102E2F00124523ED5404FDED6013124511E4FEED40
:102E3F005404FDE4FCED60057F131249B2850B19B4
:102E4F00850A18850917850816C2DF1245119008E3
:102E5F00FA12263E90086B1225F190086312263E57
:102E6F009008FA1225F1E4FFFEED5402FDE4FC9008
:102E7F00086B12263E124533603C900863124536AC
:102E8F007006900869F0A3F0900869E475F00112DC
:102E9F002356D390086AE09458900869E0648094B0
:102EAF00824046900868E070057F161249B290087C
:102EBF00687401F08033124533702E900863124509
:102ECF00366026900869E0FEA3E0FFD3940AEE6413
:102EDF00809480400FEF9458EE6480948250057F69
:092EEF00121249B2900868E4F0E7
:0A2EF800900867E004F064027067C0
:102F0200E59054039008F6F0E0FDFFE5146F5403DA
:102F12006050E514AE137802C333CE33CED8F97EB7
:102F220000540CFFED5403FDEF4D2492F582EE3474
:102F320051F583E493FF9008F7F0A3E50DF0EF2538
:102F42000DF50DE0650D30E1109008F7E0B40104D5
:102F52007F1480027F151249B29008F6E0751300C3
:072F6200F514900867E4F08C
:102F6900D007D006D005D004D003D002D001D000BC
:0B2F7900D0D0D082D083D0F0D0E03266
:10500800D2B4E4FBC2B3ED25E0FDEC33FC30B504CB
:10501800ED4401FDD2B30BEBB410E9C2B4AF05AE59
:015028000483
:015029002264
:104D0200E475F00112236C85F082F58322EEF0A3A4
:104D1200EFF0A3ECF0A3EDF0A3EAF0A3EBF022AFE7
:104D220001AE027C00E4FDA302263E08F6E4F5840F
:104D3200C2AF43B70122E0FEA3E0AA06F97B01223B
:104D7F00900954E584F0A2AF920D124D219009577E
:104D8F00E0FEA3E0781EA606124D2D438F02438F3F
:104D9F000118E6FE08E6F5828E83E4F053B7FEF5C0
:0B4DAF008FA20D92AF900954E0F58434
:014DBA0022D6
:054B190090093DEDF0E4
:104B1E00A3E584F0A2AF920E124D2190093DE0FF65
:104B2E00FD3395E0FCEDF44C6022900941E0FCA3CE
:104B3E00E0782FA604124D2D758F0118E6FC08E6BD
:104B4E00F5828C83EFF053B7FEE4F58FA20E92AF91
:064B5E0090093EE0F58421
:014B6400222E
:104BF400900943124D0F900947E07002A3E060341E
:104C0400900943124D38A3E0FEA3E0F5828E83E0C1
:104C1400FD124B1990094774FFF5F01223569009C1
:104C240045E475F001122356900943E475F001122E
:054C3400235680C2229E
:0851EF00E4900000F0A3F0229F
:104FE500900000124D38124D7F900000E0FEA3E0C6
:104FF500FF7C007D021B7A04124BF4E4900000F064
:03500500A3F022F3
:0D46E600900925EDF0900923EEF0A3EFF010
:1046F300EE54FCFE900000E0FCA3E0FD7002EE6CC3
:104703006045ED4C6003124FE5900923E0FEEE5443
:10471300FCFE7F00900000F0A3EFF0900926EEF07E
:10472300A3EFF0A37400F0A37402F07E04900926B3
:10473300124D02E493FD900928124D02EDF0EF1F94
:1047430070011EEF4E70E6900925E0FF900923E00B
:10475300FCA3E0FDEC5403FC74022DF58274003CD1
:04476300F583EFF0FB
:01476700222F
:104EC200900949124D0F90094D74FFF5F012236CB1
:104ED20045F0601A900949E475F00112236CAFF0B5
:0F4EE200FE90094B124D02E0FD1246E680D822E9
:1048DC001225FD124C399008A712263E9008A0E034
:1048EC0025E0249EF582E43407F583E0FEA3E02264
:1048FC00FBC374FF9BFF740F9EFEE49400FDE494D5
:10490C0000FC229008A0E025E02438F582E434076E
:10491C002290089FE075F00290052702267BE47F29
:10492C0001FEFDFC1225FDC3022590E47BFF7A0FEE
:0C493C00F9F8229008A71225FD02244C77
:0838A70090089FEFF0A3EDF083
:1038AF001249131248F5FBAA06E4F9F81248E8FF8B
:1038BF00E4FCFD12243E9008A312263EE49008A1DA
:1038CF00F0A3F07F0FFEFDFCA312493040089008D3
:1038DF00A1E4F0A304F074FF7FF1FEFDFC9008A3B8
:1038EF001225FDD3122590500874FF9008A1F0A364
:1038FF00F09008A1E0FEA3E0FF4E70030239FAEF4B
:07390F00F47002EEF47055A4
:1039160012490F1248F5FFE4FCFD9008AF12263E4F
:103926009008AF12492A500A9008AF12264A0000A2
:10393600000112491DE0FEA3E0FFE4FCFD12493838
:1039460012244C9008AF1248DCFFE4FCFD12493FFC
:103956009008AB12263E1249379008AB1225F11299
:023966004C39DA
:0F3968000239CF9008A1E07004A3E064017063FE
:1039770012491DE0FEA3E01248FC12493712244CFD
:103987009008A712263E12490F1248F51248FC90DC
:1039970008AB12263E9008AB12492A500A9008AB92
:1039A70012264A000000019008A71225F19008ABE3
:1039B7001248DC1248FC12493F124937124C39C3EE
:1039C70074FF9FFF740F9EFE12491DEEF0A3EFF0E8
:0339D70012513B4F
:1039DA009008A0E0FF25E0249EF582E43407F583F1
:1039EA00E0FCA3E0FDEF124913F583ECF0A3EDF040
:0139FA0022AA
:1050FD00AE05AB077F0A124A1BAF03124A1BAF0660
:06510D00124A1B0251FFD3
:0851F7007F02124A1B0251FF66
:064E6200125206EF60276A
:104E680090097D7409F0A3742AF0124F4A90097DC5
:104E7800E475F00112236C85F082F583EFF012528D
:074E88000CEF70E67F012230
:034E8F007F00227F
:0F1A2100AE077F2F124A1BAF06124A1B0251FF5E
:0F51C200AE077F30124A1BAF06124A1B0251FF85
:103C39004108FE00C105C1044708FF18100C080619
:023C4900040372
:1050D000900596E0C3135403FF2290000A12225B4E
:0750E0001313135407FF2214
:104E920090000112225BFF900983F0BFF8030239F0
:104EA200FB900983E0B4FA03025068900983E0B4EE
:0F4EB200FC030251A2900983E0B4FB031251B23A
:014EC10022CE
:10506800D205E49008FEF01250D0BF030E9005263A
:0C507800E04408F0E4FF124EF1D20422E4
:1051A200C2051250D0BF0307900526E054F7F02243
:1051B200D2051250D0BF0307900526E04408F02222
:1039FB00AF22EF3395E0FE7C007D0B1222EF748D2E
:103A0B002FF974053EFA7B019009691226B7200540
:103A1B0003023B2E9008FEE0FF04F0EFB46003744A
:103A2B0001F090096912269790000912225BC313CB
:093A3B00540364036003023B2EF6
:103A4400AF22EF3395E0FEEF25E0FFEE33FE74671F
:103A54002FF58274053EF583E0FEA3E0FFD3945B6B
:103A6400EE940F4007E490096CF08058D3EF94175C
:103A7400EE940C400890096C7401F08047D3EF94E5
:103A8400EBEE9408400890096C7402F08036D3EF92
:103A940094A7EE9406400890096C7403F08025D333
:103AA400EF94FFEE9402400890096C7404F08014C3
:103AB400D3EF9416EE940190096C40057405F080E0
:103AC400037406F09008FEE024FFFFE434FFFE9048
:103AD400096CE024FFF582E43408F583E0FD3395B6
:103AE400E0FC122301ED7042300403C2042290056D
:103AF40026E0131313541F30E030900969122697FF
:103B04001250DA64016015BF0206900716E0600CDB
:103B14001250DABF0314900716E0600E1245B47415
:0A3B2400FFF52DF52CF52B752A7F17
:013B2E002274
:023C4B00C106B0
:1040550090800275F018ED12267BEC75F018A425FA
:1040650083F8ED28AF829008DEF0A3EFF09008D634
:10407500E0FF7E007C017D181222EF74022FF97497
:10408500803EFA7BFF22E0FF75F018908002122631
:104095007BEF2583AF8222900522E475F001022390
:1040A500561222BB90096E022697900403E475F020
:1040B500011226A0AE02AF0122F9E43AFA02224229
:1040C500E024FFFFE434FFFE9008D7E0FCA3E0FD09
:1040D50022E024FFFEE434FF9008D7F0A3CEF022BF
:1040E500900522E0FCA3E0FDC39418EC940122E4C2
:1040F50075F00112236C85F082F583E49322900814
:10410500DB1226B7E49008D9F0A3F022E49005224B
:10411500F0A3F022E5C1F0A2AFE433A3F0AF05228E
:1041250074082DF58274043CF58322FE7C057D25FB
:0F4135007B187A01229FEE6480F8EC6480982258
:10513B0030000B20060A3001071251F78002D20211
:03514B00D2062267
:054DBB0090097FEFF0FC
:104DC0001251EFE4900980F090097FE0FFA3E0FE2C
:104DD000C39F501D75F018EE90800212267BEE25C1
:104DE00083AF82124130124EC2900980E004F080FD
:044DF000D7024FE5B2
:104E2D009009817402F0E4A3F01251EF7E807F00AF
:104E3D007C097D817B017A00124EC27EA07FD27CDF
:104E4D00097D827B017A00124EC2124FE5123E6936
:054E5D007F1E024DBBA9
:10509E0090A0D2E493600C908000E49364026003CD
:0950AE00124E2DE4900524F022BD
:104DF400C20690052412407578257C057D017E014C
:104E04007F181221FAE4FF75F00BEF900595122636
:104E14007BE0C4135401FE74172FF582E43407F5C4
:084E240083EEF00FEFB410DF84
:014E2C002263
:105160001251EF90052412408B124130124EC202B0
:025170004FE509
:061A3300125160C2062200
:0A42FB009008D3EDF09008D2EFF028
:10430500D39B40321240D6EB149008D6F09008D3D8
:104315001240C5D312413A5057124055124103126B
:10432500437640FB124FE59008D712409F9008D680
:10433500E004F00243129008D31240D69008D5E06D
:1043450014A3F09008D21240C5C312413A4021127D
:10435500405512410312437640FB124FE59008D7B2
:1043650074FFF5F01223569008D6E014F002434886
:10437500229008DBE475F0011226A0AE02AF019091
:1043850008DEE475F00112236C85F082F583E49371
:10439500FD1246E69008D9E475F001122356C39044
:0C43A50008DAE094189008D9E094012296
:0543B100900402EDF094
:1043B600EF14900520F0EB14A3F0900402E014FF34
:1043C600900520E0D39F4003024466A312408BFE73
:1043D6001241111240E550190FEFAA0670010E1492
:1043E600F5828A83E493FB124125EBF012409C8010
:1043F600E29005211240759004031226B79005201D
:1044060012408B900406F0A3EFF01241111240AF58
:104416009004061240F4FD1246E612409CC3900535
:1044260023E09418900522E0940140E190052012C3
:1044360040759004031226B71241111240E5501040
:104446001240AF124125E0FD1246E612409C80EB79
:10445600124FE5900520E004F0A3E004F00243C00B
:014466002233
:074467009008EBEBF0AC073D
:10446E00A3124119A3E4F0A3EFF0E07F00FE900841
:10447E00EEF0A3EFF0AD04EDFF9008EEEEF0A3EF3B
:10448E00F020C7FD20C3FAC2AF900524740FF012BE
:10449E0051EF9005241240759008F21226B7E49061
:1044AE0008F0F0A3F09008EEE0FCA3E0FFECFD9026
:1044BE0008EBE0FBE4900974F0D208124144900836
:1044CE00F5EFF0FD9008F21240B21246E69008EEBB
:1044DE0012409F9008F012409FC39008F1E094188C
:1044EE009008F0E0940140BD124FE5900524E004E1
:1044FE00F0E0C3941E4098124D429008EDE024FF68
:02450E0092AF6A
:014510002288
:04464E00AC07AA0308
:1046520090090612411990090AE4F0A3EFF0E0F87C
:10466200E4F0E890090AF0AF04E0F0A3E04FF02094
:10467200C7FD20C3FAC2AF900524740FF090052441
:10468200E0FFC3941E505175F018EF12409090094C
:104692000CF0A3EFF0E4900908F0A3F090090AE00F
:1046A200FCA3E0FFECFDAB02A31240F4900974F00E
:1046B200C20812414490090A12409F900908124010
:1046C2009FC3900909E09418900908E0940140CC36
:1046D200900524E004F080A5124D42900907E024E1
:0346E200FF92AF95
:0146E50022B2
:103E6900E4900525F0A3E054F8F054F7F0E4900944
:103E79006DF090096DE0FFC39433501675F002EFB1
:103E890090052712267BE4F0A3F090096DE004F079
:103E990080E09005877408F0A3E4F090096DF09034
:0C3EA900096DE0FFC394104003023F626B
:103EB500EF75F00BA4248DF9740535F0FA7B01A399
:103EC5001226B71240A9E41240A6900001E412227E
:103ED500CD900002E4F5F0122404900004E41222CF
:103EE500CD900005E41222CDE924061240BE54C04F
:103EF5001240A6E924071240BE54F81222BB54C74B
:103F05001240A6E924081240BE54F81222BB54F709
:103F15001222BB54EF1222BB54DF1222BB54BF1234
:103F250022BB547F1240A6E924091240BE54FE125A
:103F350022BB54F944021222BB54C744281240A69E
:103F4500E9240A1240BE54F844051222BB54C74462
:043F5500081222BB71
:093F590090096DE004F0023EA89D
:013F6200223C
:07414400900971EFF0A905DD
:10414B00C20920C3FD20C5FAC2C4D2C5E4FFFD30AD
:10415B00C3FD30C3FDE5C154F8FC64086004ECB446
:10416B001013EFB40105EB44018003EB54FEF5C2D1
:10417B007D01024212ECB4180B89C27D02C2C4C28B
:10418B00C5024212ECB420028045EC6428703CED71
:10419B00B4020E900971E0F5C27D03C2C5C2C480A2
:1041AB0066EDB4031B300808D2C57F01C2C480572B
:1041BB00900974E0F5C2C2C57D04E4FFC2C4804718
:1041CB00ED64047042D2C47D05803CECB4300AD25D
:1041DB00C4D2C57D08E4FF802EECB438028024ECF9
:1041EB00B44006C2C2C2C5801EECB448028014ECB7
:1041FB00B450028004ECB4580AD2C47D07AEC2C2DC
:10420B00C28004D2C4D2C5C2C3ED64076008ED649A
:08421B0005600302415DAF06DE
:014223002278
:083C4D0041080C0041082500AC
:104CC00090080FE475F00112236C85F082F58322C1
:104CD00090080F7408F0A37426F022900808E47579
:104CE000F0011223567E087F3A900808E0229008CF
:104CF0000AE0FFA3E090080822E0F5C2900808E06F
:024D00006E2221
:1050B700AF84E4F584C2C343E60243F60275C30135
:0850C70075C04475CF8F8F8482
:0150CF0022BE
:104D42007E087F11900806EEF0A3EFF090080DEEBA
:104D5200F0A3EFF0900804EEF0A3EFF07E087F26B8
:104D620090080AEEF0A3EFF090080FEEF0A3EFF038
:0D4D7200900808EEF0A3EFF0C20A0250B75F
:104F9B0090080D124CC3EFF090080D124CC3EDF0BE
:104FAB0090080DE0B4080FA3E0B4250A90080D7427
:074FBB0008F0A37411F022BD
:0751FF00C20AC2C4D2C5229E
:104A1B00200A2FD20A124CC074FFF07C087D3A900A
:104A2B00080FE0B50408A3E0B50503124CD0124CF7
:104A3B00C0E4F090080FE0B50408A3E0B50503123D
:104A4B004CD0124CC0E4F090080FE0B40808A3E07F
:104A5B00B43A03124CD0124CC0EFF090080FE0B4F4
:0D4A6B000808A3E0B43A03124CD07F0122EA
:104F1E00900806E0FCA3E0FD900804E0B50408A3A9
:104F2E00E0B505037F0022900806E0FCA3E0F582C1
:0C4F3E008C83E0B507037F01227F002276
:104F4A00900806E475F001122356900806124CC325
:104F5A00E0FF900806E0B4080FA3E0B4250A900821
:084F6A00067408F0A37411F0B5
:014F7200221C
:065206007FFF124F1E2283
:06520C00E4FF124F1E2218
:031A18000233D2C4
:1033D200C0E0C0F0C083C082C0D075D000C000C0C1
:1033E20004C005C006C007E5C154F81226C0354620
:1033F20000342D08342D10345618347D203483289F
:1034020034E33034E83834F75034F7583503603455
:10341200F96835037034F97834F780351B8834F74E
:1034220090351B98352EA000003573C2C5124CDBB7
:10343200B5060BA3E0B50706900808124CD3900816
:1034420008124CC3124CF97003A3E06F60030235FB
:10345200730234DA124CDBB5060BA3E0B507069013
:103462000808124CD3900808124CC3124CF970038E
:10347200A3E06F60030235730234DA124CEECF80A0
:103482001990080FE0FEA3E0FF900808E0FCA3E01B
:10349200FDB50711ECB5060DA3EEF0A3EFF0C2C522
:1034A200D2C40235738D828C83E0B4FF07C2C4D2CA
:1034B200C5023573124CDBB5060BA3E0B5070690C7
:1034C2000808124CD3900808124CC3124CF970032E
:1034D200A3E06F6003023573900808124CD30235E3
:1034E20073124CEE803D124CEECFF0A3EFF0D2C43B
:1034F200D2C50235738019124CEECFF0A3EFF0D291
:103502000BADC27FFF124F9B90080C7401F08061DB
:10351200ADC2E4FF124F9B8058900804E0FFA3E085
:1035220090080DCFF0A3EFF0D2C4804590080DE0D3
:10353200FFA3E0900804CFF0A3EFF0300B33D2C525
:10354200C20B802D90080AE0FEA3E0FF900808EE6F
:10355200F0A3EFF0900804E0FDA3E090080DCDF099
:10356200A3EDF0D2C4A3E06E7003A3E06F6002D2B9
:10357200C5C2C3D007D006D005D004D000D0D0D069
:0835820082D083D0F0D0E032CA
:03000000020C00EF
:03000300021A03DB
:03000B00021A06D0
:03001300021A09C5
:03001B00021A0CBA
:03002300021A0FAF
:03002B00021A12A4
:03003300021A1599
:03003B00021A188E
:03004300021A1B83
:03004B00021A1E78
:03005300021A216D
:03005B00021A2462
:03006300021A2757
:03006B00021A2A4C
:03007300021A2D41
:03007B00021A3036
:03008300021A332B
:03008B00021A3620
:03009300021A3915
:03009B00021A3C0A
:0300A300021A3FFF
:100C0000787FE4F6D8FD9000007F007E20E4F0A31A
:0A0C1000DFFCDEFA758130020C559E
:100C1A00021A3CE493A3F8E493A34003F68001F29A
:100C2A0008DFF48029E493A3F85407240CC8C333DB
:100C3A00C4540F4420C8834004F456800146F6DFAA
:100C4A00E4800B0102040810204080903B2FE47ED0
:100C5A00019360BCA3FF543F30E509541FFEE4939F
:100C6A00A360010ECF54C025E060A840B8E493A366
:100C7A00FAE493A3F8E493A3C8C582C8CAC583CA91
:100C8A00F0A3C8C582C8CAC583CADFE9DEE780BE49
:013C5500006E
:10212A00E709F608DFFA8046E709F208DFFA803E97
:10213A0088828C83E709F0A3DFFA8032E309F60884
:10214A00DFFA8078E309F208DFFA807088828C83EC
:10215A00E309F0A3DFFA806489828A83E0A3F608A0
:10216A00DFFA805889828A83E0A3F208DFFA804C7A
:10217A0080D280FA80C680D4806980F28033801051
:10218A0080A680EA809A80A880DA80E280CA8033BA
:10219A0089828A83ECFAE493A3C8C582C8CCC58332
:1021AA00CCF0A3C8C582C8CCC583CCDFE9DEE78002
:1021BA000D89828A83E493A3F608DFF9ECFAA9F081
:1021CA00EDFB2289828A83ECFAE0A3C8C582C8CCD7
:1021DA00C583CCF0A3C8C582C8CCC583CCDFEADEF0
:1021EA00E880DB89828A83E493A3F208DFF980CC52
:1021FA0088F0EF60010E4E60C388F0ED2402B4044B
:10220A000050B9F582EB2402B4040050AF232345F1
:06221A00822390217A737B
:10222000C2D530F707B2D563F0FF05F030E70CB246
:10223000D5F4048463F0FF05F080018430D502F406
:02224000042276
:10224200BB010689828A83E0225002E722BBFE029A
:09225200E32289828A83E49322CD
:10225B00BB010CE58229F582E5833AF583E0225038
:10226B0006E92582F8E622BBFE06E92582F8E22282
:0D227B00E58229F582E5833AF583E493229C
:10228800BB010FF8E58229F582E5833AF583E0285A
:10229800F0225009C58229F8E58226F622BBFE09FC
:1022A800C58229F8E22582F222F8EA2583F583E936
:0322B80093282246
:1022BB00BB010689828A83F0225002F722BBFE0102
:0222CB00F322FC
:1022CD00F8BB010DE58229F582E5833AF583E8F047
:1022DD00225006E92582C8F622BBFE05E92582C8F3
:0222ED00F222DB
:1022EF00EF8DF0A4A8F0CF8CF0A428CE8DF0A42E03
:0222FF00FE22BD
:10230100BC000BBE0029EF8DF084FFADF022E4CCC0
:10231100F875F008EF2FFFEE33FEEC33FCEE9DEC89
:10232100984005FCEE9DFE0FD5F0E9E4CEFD22EDCF
:10233100F8F5F0EE8420D21CFEADF075F008EF2F19
:10234100FFED33FD4007985006D5F0F222C398FD0A
:052351000FD5F0EA22A7
:10235600C5F0F8A3E028F0C5F0F8E5821582700212
:062366001583E038F022AF
:10236C00A3F8E0C5F025F0F0E58215827002158324
:06237C00E0C838F0E82281
:10238200BB010A89828A83E0F5F0A3E02250068726
:10239200F009E71922BBFE07E3F5F009E3192289E8
:0B23A200828A83E493F5F0740193221B
:1023AD00BB0110E58229F582E5833AF583E0F5F06E
:1023BD00A3E0225009E92582F886F008E622BBFE4B
:1023CD000AE92582F8E2F5F008E222E5832AF58391
:0823DD00E993F5F0A3E9932256
:1023E500BB010A89828A83F0E5F0A3F0225006F743
:0F23F50009A7F01922BBFE06F3E5F009F3192240
:10240400F8BB0111E58229F582E5833AF583E8F00A
:10241400E5F0A3F0225009E92582C8F608A6F022C7
:0D242400BBFE09E92582C8F2E5F008F222AE
:0D243100EF2BFFEE3AFEED39FDEC38FC22FA
:0E243E00C3EF9BFFEE9AFEED99FDEC98FC2299
:10244C00E88FF0A4CC8BF0A42CFCE98EF0A42CFC2F
:10245C008AF0EDA42CFCEA8EF0A4CDA8F08BF0A4AD
:10246C002DCC3825F0FDE98FF0A42CCD35F0FCEB0C
:10247C008EF0A4FEA9F0EB8FF0A4CFC5F02ECD39D1
:0F248C00FEE43CFCEAA42DCE35F0FDE43CFC223E
:10249B0075F008758200EF2FFFEE33FECD33CDCCF8
:1024AB0033CCC58233C5829BED9AEC99E58298407B
:1024BB000CF582EE9BFEED9AFDEC99FC0FD5F0D658
:1024CB00E4CEFBE4CDFAE4CCF9A88222B800C1B982
:1024DB000059BA002DEC8BF084CFCECDFCE5F0CBC0
:1024EB00F97818EF2FFFEE33FEED33FDEC33FCEBF9
:1024FB0033FB10D703994004EB99FB0FD8E5E4F9B4
:10250B00FA227818EF2FFFEE33FEED33FDEC33FCA0
:10251B00C933C910D7059BE99A4007EC9BFCE99A94
:10252B00F90FD8E0E4C9FAE4CCFB2275F010EF2FD9
:10253B00FFEE33FEED33FDCC33CCC833C810D707D9
:10254B009BEC9AE899400AED9BFDEC9AFCE899F814
:0E255B000FD5F0DAE4CDFBE4CCFAE4C8F922A7
:104C3900C2D5E830E70FB2D5E4C39BFBE49AFAE4A6
:104C490099F9E498F8EC30E717B2D5124C6F1224B1
:104C5900D7E4C39BFBE49AFAE499F9E498F8800352
:104C69001224D730D50DE4C39FFFE49EFEE49DFDD9
:044C7900E49CFC2299
:0D256900EF5BFFEE5AFEED59FDEC58FC2231
:0D257600EF4BFFEE4AFEED49FDEC48FC2264
:0D258300CFF4CFCEF4CECDF4CDCCF4CC22ED
:10259000EB9FF5F0EA9E42F0E99D42F0EC6480C8C2
:0625A00064809845F02262
:1025A600EB9FF5F0EA9E42F0E99D42F0E89C45F08B
:0125B6002202
:1025B700E8600FECC313FCED13FDEE13FEEF13FF02
:0325C700D8F12226
:1025CA00E86010ECA2E713FCED13FDEE13FEEF1327
:0425DA00FFD8F02214
:1025DE00E8600FEFC333FFEE33FEED33FDEC33FC5B
:0325EE00D8F122FF
:0C25F100E0FCA3E0FDA3E0FEA3E0FF225D
:0C25FD00E0F8A3E0F9A3E0FAA3E0FB2261
:102609007401FF3395E0FEFDFCA3A3A3E0CF2FF0F7
:10261900E582158270021583E0CE3EF0E5821582CF
:1026290070021583E0CD3DF0E582158270021583B5
:05263900E0CC3CF022A2
:0C263E00ECF0A3EDF0A3EEF0A3EFF0220F
:10264A00A8828583F0D083D0821226611226611275
:10265A002661122661E473E493A3C583C5F0C5839A
:10266A00C8C582C8F0A3C583C5F0C583C8C582C8DA
:01267A00223D
:0C267B00A42582F582E5F03583F583226A
:10268700FAE6FB0808E6F925F0F618E6CA3AF62254
:09269700E0FBA3E0FAA3E0F92244
:1026A000F8E0FBA3A3E0F925F0F0E58215827002C3
:0726B0001583E0FA38F02267
:0926B700EBF0A3EAF0A3E9F02224
:1026C000D083D082F8E4937012740193700DA3A3A9
:1026D00093F8740193F5828883E4737402936860BD
:0626E000EFA3A3A380DFBD
:00000001FF
